:0200000480007A
:100000006F008004732F2034930F80006308FF0378
:10001000930F90006304FF03930FB0006300FF038E
:10002000130F000063040F0067000F00732F2034CC
:1000300063540F006F00400093E19153171F0000BD
:1000400023223FFC6FF09FFF732540F163100500F2
:10005000970200009382020173905230735000188F
:10006000970200009382020273905230B702008020
:100070009382F2FF7390023B9302F0017390023A75
:1000800097020000938282017390523073502030A7
:1000900073503030735040309301000097020000DD
:1000A000938282F673905230130510001315F501F8
:1000B000634C05000F00F00F930110009308D0056A
:1000C000130500007300000093020000638E02001D
:1000D00073905210B7B20000938292107390223046
:1000E00073232030E39A62F47350003097020000CB
:1000F0009382420173901234732540F173002030D3
:10010000B710FF00938000F013C7F0F0B7FE00FFB8
:10011000938EFE00930120006316D71DB710F00FD9
:10012000938000FF13C7000FB71EF00F938E0EF0E1
:10013000930130006318D71BB710FF009380F08F36
:1001400013C7F070B71EFF00938E0EFF930140009F
:10015000631AD719B7F00FF09380F00013C7000FA0
:10016000B7FE0FF0938EFE0F93015000631CD7175C
:10017000B7F000FF9380007093C0F070B7FE00FFEF
:10018000938EFE0093016000639ED0151302000061
:10019000B710F00F938000FF13C7000F1303070081
:1001A0001302120093022000E31452FEB71EF00F58
:1001B000938E0EF0930170006316D31313020000A8
:1001C000B710FF009380F08F13C7F070130000008A
:1001D000130307001302120093022000E31252FEE1
:1001E000B71EFF00938E0EFF93018000631CD30F98
:1001F00013020000B7F00FF09380F00013C7000F58
:100200001300000013000000130307001302120084
:1002100093022000E31052FEB7FE0FF0938EFE0F04
:10022000930190006310D30D13020000B710F00F7C
:10023000938000FF13C7000F1302120093022000E7
:10024000E31652FEB71EF00F938E0EF09301A0003E
:10025000631AD70913020000B710FF009380F0FF64
:100260001300000013C7F0001302120093022000D5
:10027000E31452FEB71EFF00938E0EFF9301B000F1
:100280006312D70713020000B7F00FF09380F0005D
:10029000130000001300000013C7000F1302120028
:1002A00093022000E31252FEB7FE0FF0938EFE0F72
:1002B0009301C0006318D7039340000F930E000F03
:1002C0009301D0006390D003B700FF009380F00F3C
:1002D00013C0F070930E00009301E0006314D0018E
:1002E000631030020F00F00F638001009391110042
:1002F00093E111009308D0051385010073000000FD
:100300000F00F00F930110009308D00513050000B3
:1003100073000000731000C0000000000000000027
:1003200000000000000000000000000000000000CD
:0C033000000000000000000000000000C1
:1010000000000000000000000000000000000000E0
:1010100000000000000000000000000000000000D0
:1010200000000000000000000000000000000000C0
:1010300000000000000000000000000000000000B0
:081040000000000000000000A8
:040000058000000077
:00000001FF
